:100000000C9434000C9451000C9451000C94510049
:100010000C9451000C9451000C9451000C9451001C
:100020000C9451000C9451000C9451000C9451000C
:100030000C9451000C9451000C9451000C945100FC
:100040000C9451000C9451000C9460040C945100D9
:100050000C9451000C9451000C9451000C945100DC
:100060000C9451000C94510011241FBECFEFD8E026
:10007000DEBFCDBF16E0A0E0B1E0EEE8FBE102C0DC
:1000800005900D92A03AB107D9F727E0A0EAB6E0B3
:1000900001C01D92A432B207E1F70E94DC030C9468
:1000A000C50D0C940000F999FECF92BD81BD60BDD5
:1000B000FA9AF99A0895F999FECF92BD81BDF89AFE
:1000C00080B50895EF92FF920F931F93CF93DF9324
:1000D0008C01EB017B01E40EF51ECE15DF0539F036
:1000E0006991C8010E9453000F5F1F4FF6CFDF9147
:1000F000CF911F910F91FF90EF900895EF92FF9293
:100100000F931F93CF93DF938B01040F151FEB0108
:100110007C01E61AF70AC017D10739F0C7018C0F26
:100120009D1F0E945B008993F6CFDF91CF911F91B5
:100130000F91FF90EF9008956F927F928F929F9210
:10014000AF92BF92CF92DF92EF92FF920F931F93E5
:10015000CF93DF93CDB7DEB7C254D1090FB6F89471
:10016000DEBF0FBECDBF6C018B017A0143E050E0D2
:1001700060E071E0C8010E94900A892B09F080C0FC
:10018000F8018381882309F47BC040E150E070E0EE
:1001900060E0C80104960E94530923967FAF6EAFBA
:1001A00023976115710509F465C0860100561F4F3C
:1001B000F8015081503208F05DC09B0145E065E2D6
:1001C00070E0C601F5E05F9F800D911D11240E9433
:1001D000D206F80160816F5F90E080E00E945300DA
:1001E000F801808190E0880F991F42E050E0BE0145
:1001F0006F5B7F4F01960E94620023968FAD23971D
:100200008F9322968FAD22978F93F80180811F9252
:100210008F9384E091E09F938F939E012F5F3F4FD8
:1002200069013F932F930E94A60A40E450E0B60173
:10023000C7010E94A204F80180818F5F80830FB6FE
:10024000F894DEBF0FBECDBFCE5BDF4F0FB6F89484
:10025000DEBF0FBECDBFDF91CF911F910F91FF90F9
:10026000EF90DF90CF90BF90AF909F908F907F9056
:100270006F90089564E271E0C7010E94BE04E4CF6C
:1002800044E050E06DE571E0C8010E94900A892BBE
:10029000D1F562E671E0C7010E94BE04712C4601EF
:1002A00030EA830E911C85E0682E91E1A92E91E041
:1002B000B92E8E010F5F1F4FF40180817816F0F484
:1002C000C601769C800D911D11240E94CE069F933D
:1002D0008F931F927F92BF92AF921F930F930E94B2
:1002E000A60A40E450E0B801C7010E94A20473943A
:1002F0000FB6F894DEBF0FBECDBFDECF6AE0C701F8
:100300000E949B04A1CF42E050E066E872E0C80181
:100310000E94900A892BB1F5F8018281882391F11E
:10032000C80102960E94690AF601E056FF4F20813B
:10033000281728F18C011127960145E0849F200D94
:10034000311D1124C9010E9494061F930F938BE65F
:1003500091E09F938F938E010F5F1F4F1F930F9319
:100360000E94A60A40E450E0B801C7010E94A2041E
:100370000F900F900F900F900F900F9065CF60E847
:1003800071E07ACF43E050E06EE972E0C8010E946C
:10039000900A892BF1F4F80183818823D1F0C801F8
:1003A00003960E94690AF601E056FF4F2081281744
:1003B00030F38C011127960145E0849F200D311DFB
:1003C0001124C9010E94B1061F930F9380E991E0A7
:1003D000C0CF4BE150E0B801C7010E94A20466EA19
:1003E00071E04ACFAF92BF92CF92DF92EF92FF922D
:1003F0000F931F93CF93DF93CDB7DEB7C054D109CE
:100400000FB6F894DEBF0FBECDBF6C018B017A0131
:1004100042E050E066E872E0C8010E94900A892B31
:1004200049F4C6010E945B076BED71E0C7010E94B1
:10043000BE043FC043E050E06EE972E0C8010E9494
:10044000900A892B31F4C6010E9486076AEE71E09A
:10045000EDCF45E050E06AEF71E0C8010E94900ADC
:10046000892BC9F5C6010E944809082FC6010E94C0
:100470004B09182FC6010E9446091F920F931F9225
:100480001F931F928F9380E092E09F938F938E0132
:100490000F5F1F4F1F930F930E94A60A40E450E086
:1004A000B801C7010E94A2040FB6F894DEBF0FBEC8
:1004B000CDBFC05CDF4F0FB6F894DEBF0FBECDBF1F
:1004C000DF91CF911F910F91FF90EF90DF90CF9030
:1004D000BF90AF90089543E050E061E772E0C8013B
:1004E0000E94900A892B41F5F80180E091919923AF
:1004F00021F08C3139F08F5FF9CF67E372E08F30F4
:1005000008F494CFF80117821386C8010C960E9454
:10051000690AA82EC80108960E94690AB82EC80167
:1005200004960E94690A2A2D4B2D682FC6010E944D
:10053000930767E272E07ACF47E050E069E572E046
:10054000C8010E94900A892B59F4C80108960E949C
:10055000690A682FC6010E94680761E672E066CFEB
:1005600046E050E06EE672E0C8010E94900A892BD6
:1005700059F4C80107960E94690A682FC6010E94B3
:10058000A70765E772E052CF47E050E061E872E00C
:10059000C8010E94900A892B39F461E0C6010E94CB
:1005A000F90769E872E042CF48E050E069E972E09B
:1005B000C8010E94900A892B39F460E0C6010E94AC
:1005C000F90762EA72E032CF4CE150E0B801C701AE
:1005D0000E94A20463EB72E029CFAF92BF92CF9248
:1005E000DF92EF92FF920F931F93CF93DF93CDB7DC
:1005F000DEB7A0970FB6F894DEBF0FBECDBF8C015B
:100600006B015A010E94E204882301F140E250E0AC
:10061000BE016F5F7F4FC8010E9424057C01892BBA
:10062000A9F085E0E816F10414F145E050E067EF29
:1006300072E0CE0101960E94900A892BE1F4A80194
:10064000BE01695F7F4FC6010E949C00A0960FB655
:10065000F894DEBF0FBECDBFDF91CF911F910F91F8
:10066000FF90EF90DF90CF90BF90AF90089583E020
:10067000E816F104BCF143E050E06DEF72E0CE010A
:1006800001960E94900A892B41F4A801BE016B5F7C
:100690007F4FC5010E94F201D9CF85E0E816F10431
:1006A0000CF145E050E061E073E0CE0101960E945C
:1006B000900A892BB9F4F12CE12C60E0C7010E946B
:1006C00053008FEFE81AF80A81E4E816F104A9F75D
:1006D00067E073E0C8010E94BE04F601E056FF4FD8
:1006E0001082B4CF89818F3371F084E0E816F10471
:1006F00084F044E050E066E173E0CE0101960E9490
:10070000900A892B31F46BE173E0C8010E94BE04AA
:100710009DCF6DE676E0F9CFCF92DF92EF92FF9218
:100720000F931F93CF93DF9300D0CDB7DEB76C014B
:1007300090E080E00E945B00760190EAE90EF11CF7
:10074000F7018083813268F010E000E060E0C801CA
:100750000E9453000F5F1F4F01341105B9F7F701D5
:10076000108210E005E0F70180818117D0F0812F21
:1007700090E0880F991F42E050E0BE016F5F7F4F0D
:1007800001960E947E0029813A8145E065E270E091
:10079000C601109F800D911D11240E94D2061F5F7B
:1007A000E2CF0F900F90DF91CF911F910F91FF90AB
:1007B000EF90DF90CF900895CF93DF93CDB7DEB762
:1007C000C15CD1090FB6F894DEBF0FBECDBF82E287
:1007D00084B988E68AB915B87894CE0181549F4FC0
:1007E0000E9486041F92812CAA24A394CC24C39433
:1007F00083E0E82E08E410E027E430E045E450E030
:1008000064E470E0CE0189549F4F0E94DA061F9283
:10081000C12C95E0E92E04EB10E023EB30E041EB36
:1008200050E060EB70E0CE0181559F4F0E94DA06E8
:10083000CE0189549F4F0E941F07CE0181559F4FC3
:100840000E941F07AE0141555F4FBE0169547F4FA3
:10085000CE018E559F4F0E944A078E010F5F1F4F9A
:100860006E0181EAC80ED11C0F900F907801C8016B
:100870000E94D9060B5F1F4F0C151D05C1F7F8012B
:100880001082C7010E948C0362E876E0CE01815499
:100890009F4F0E94BE04AE014E555F4FB701CE017F
:1008A00081549F4F0E94ED02CE018E559F4F0E94B2
:1008B000CC088FE39FE10197F1F700C00000EBCF78
:1008C0001F920F920FB60F9211248F939F93EF9365
:1008D000FF938091C600E091A006F091A106EF770A
:1008E000FF27EE55F94F80838091A0069091A106D5
:1008F00001969093A1068093A006FF91EF919F919E
:100900008F910F900FBE0F901F9018952AE0FC0159
:100910002083128211821092C50089E18093C40065
:1009200086E08093C200E1ECF0E088E18083808182
:100930008068808308958091C00085FFFCCF60931C
:10094000C6000895EF92FF920F931F93CF93DF930A
:100950007C01EB018B01040F151FC017D10739F083
:100960006991662321F0C7010E949B04F6CFDF91B5
:10097000CF911F910F91FF90EF900895EF92FF920A
:100980000F931F93CF93DF937C01EB018B01FE014B
:1009900001900020E9F73197EC1BFD0BC8018C1B7F
:1009A0009D0B8E179F0738F4F80161918F01C701E5
:1009B0000E949B04ECCFDF91CF911F910F91FF908C
:1009C000EF9008954091A0065091A10621E0FC010E
:1009D000818192818417950708F020E0822F089585
:1009E000FC01128211821092A1061092A006E2EA86
:1009F000F6E080E2819397E0E232F907D9F70895B3
:100A0000CF93DF93EC0189819A8181159F4718F07C
:100A1000CE010E94F00489819A812091A006309134
:100A2000A1068217930770F49C012F5F3F4F3A8312
:100A300029838F779927FC01EE55F94F8081DF914B
:100A4000CF91089580E0FBCF8F929F92AF92BF929B
:100A5000CF92DF92EF92FF920F931F93CF93DF938A
:100A60008C016B01FC0181819281D0E0C0E020917A
:100A7000A0063091A106281B390B2C173D0788F0E2
:100A8000C138D10571F0FC01EC0FFD1FEF77FF2796
:100A9000EE55F94F3081F8012081321711F021967F
:100AA000E6CF2091A0063091A106281B390BC21772
:100AB000D30710F4209739F481159F4708F043C0FD
:100AC000D0E0C0E020C04601F12CE12C5A0121E029
:100AD000A21AB108EA14FB0464F4C8010E940005DC
:100AE000F40181934F01FFEFEF1AFF0ACE15DF05E6
:100AF00089F7EC0CFD1CF7011182F80181819281CC
:100B0000019692838183F80181819281FC01EC0F2F
:100B1000FD1FEF77FF27EE55F94F3081F801208157
:100B2000321303C0019692838183CE01DF91CF916E
:100B30001F910F91FF90EF90DF90CF90BF90AF90FB
:100B40009F908F900895C8010E94F004B9CFDC01F6
:100B50001296ED91FC91139714968C91149721E0C5
:100B600030E0A90101C0440F8A95EAF7942F9095CF
:100B70008081892380838081842B8083613009F088
:100B80004DC087EE93E00197F1F700C00000129688
:100B9000ED91FC911397408114968C911497B901B3
:100BA00002C0660F771F8A95E2F7CB0180958423F8
:100BB000808387EB9BE00197F1F700C0000012965D
:100BC000ED91FC911397808114969C911497A90143
:100BD00001C0440F9A95EAF7942F9095982390833B
:100BE0008081842B808387EE93E00197F1F700C02A
:100BF00000001296ED91FC911397808114969C91C0
:100C000001C0220F9A95EAF720952823208387EBCD
:100C10009BE00197F1F700C00000089587EB9BE08F
:100C20000197F1F700C000001296ED91FC91139727
:100C3000808114969C911497A90101C0440F9A9544
:100C4000EAF740954823408387EE93E00197F1F758
:100C5000B4CFEF92FF920F931F93CF93DF93EC01EA
:100C6000EA81FB8120813C8181E090E0AC0101C000
:100C7000440F3A95EAF7342F3095322330832081A0
:100C8000242B2083E7EEF3E03197F1F700C000005A
:100C9000EA81FB8120813C8101C0880F3A95EAF707
:100CA00080958223808387EB9BE00197F1F700C05A
:100CB00000000FE010E0EE24E394F12C288139814C
:100CC000C701002E02C0880F991F0A94E2F7822301
:100CD000932361E0892B09F460E0CE010E94A7050F
:100CE000015011090530110549F7DF91CF911F918E
:100CF0000F91FF90EF900895DC011296ED91FC9119
:100D00001397208114963C9181E090E001C0880FF8
:100D10003A95EAF780958223808387E199E70197E6
:100D2000F1F700C0000008950F931F93CF93DF9356
:100D3000EC010AE010E0CE010E94290661E0CE013C
:100D40000E94A70560E0CE010E94A705CE010E9487
:100D50007C060150110979F7DF91CF911F910F9116
:100D600008950F931F93CF93DF93EC010AE010E0F7
:100D7000CE010E94290660E0CE010E94A70561E035
:100D8000CE010E94A705CE010E947C0601501109E8
:100D900079F7DF91CF911F910F910895FC01808128
:100DA00091810895FC01738362833183208344839E
:100DB00008950895AF92CF92EF920F931F93CF9320
:100DC000DF93CDB7DEB7FC01718360833383228369
:100DD00015830483C682A782DB011C92DA011C9270
:100DE0008681882331F020813181D9018C918068FE
:100DF0008C938781882331F020813181D9018C91B6
:100E000080628C9320813181D9018C9183608C9395
:100E1000DA018C91BE2DB770EB2EE82ADA01EC9244
:100E2000A281B3811C920480F581E02D1082DF91B4
:100E3000CF911F910F91EF90CF90AF900895DC016B
:100E4000ED91FC918081837080830895CF93DF932F
:100E5000EC010E941F078E81882329F0E881F98127
:100E60008081806880838F81882329F0E881F981DF
:100E7000808180628083DF91CF910895DC0112969A
:100E8000ED91FC9160830895DC011496ED91FC9145
:100E900060830895FC0171836083538342831482CD
:100EA00016821582178210861186128681E083874A
:100EB00087E084870895CF93DF93EC01888199813F
:100EC0000E9426078A819B81DF91CF910C9426078F
:100ED000CF93DF93EC016C836623A9F060E08881F7
:100EE00099810E94440760E0888199810E943E07B1
:100EF00060E08A819B810E944407CE010E945B07CB
:100F00001F821E821D82DF91CF910895CF93DF93C0
:100F1000EC01888199810E941F078A819B81DF9162
:100F2000CF910C941F07FC011482608741872287B0
:100F3000338531110AC0620F7727771F460F572F6D
:100F4000511D452B11F40C9486070C945B076150DE
:100F5000603108F04BC0E62FF0E0EF54F84F0C94EE
:100F60004D09C107C607CA07CE07D207D507D8075C
:100F7000DB07DE07DB07E207E607EA07EE07F20713
:100F8000F40720E54FEF60EA0C94930724E14FEF5C
:100F900068ECFACF2CE84FEF64EBF6CF20E040E0AE
:100FA0006FEFF2CF2AE04CE3FBCF2EE14EE1F8CF1A
:100FB00020E04BE9F5CF20E04FEF0AC02AE04FEFE9
:100FC00067E3E2CF27E040E568E0DECF2FEF40E0C7
:100FD00060E0DACF2FEF4FEF62E3D6CF26E940E5AE
:100FE0006AE0D2CF2CEDE8CF20E0D1CF24E14DE272
:100FF000D7CFFC0163870895CF93DF93EC018C81F9
:10100000813041F58D819E812F8121111CC0019677
:101010009E838D836D817E816F3F7105B1F481E088
:101020008F83888199810E9444076D8160958881B2
:1010300099810E943E076D8160548A819B81DF9176
:10104000CF910C9444070197E3CF6115710549F7DF
:101050001F82E7CF823021F58D819E812F81211162
:1010600018C001969E838D836D817E816E3F21E045
:10107000720789F481E08F837695679588819981DD
:101080000E94440760E0888199810E943E0760E0E9
:10109000D4CF0197E7CF6115710571F71F82ECCFAF
:1010A000833069F58D819E812F81211121C00196A8
:1010B0009E838D836D817E8161158FEF7807D1F4DA
:1010C00081E08F8346E0769567954A95E1F78881C0
:1010D00099810E9444076E81888199810E943E0710
:1010E0006D817E8153E0769567955A95E1F7A5CF9E
:1010F0000197DECF6115710529F71F82E3CF843098
:10110000F1F56D817E8188819981611520E27207F8
:10111000C8F536E0769567953A95E1F70E94440761
:101120006D817E81613080E2780770F088819981DD
:10113000611520E4720760F5705226E07695679598
:101140002A95E1F70E943E076D817E81613080E43F
:10115000780768F064E0769F612D7727112484E199
:10116000689F602D11248A819B810E9444078D8194
:101170009E818F3F980719F001969E838D83DF91A2
:10118000CF910895672F6695669566956058C6CF8E
:10119000672F66956058D6CFCF93DF93EC010E94FE
:1011A000FC078C8181116FC08B85882309F45FC097
:1011B0008D819E8101969E838D839C8501C0880FC1
:1011C0009A95EAF781115FC098B588858917B1F0C3
:1011D00068B528B5281B330B81E090E01216130682
:1011E00014F090E080E0232F221F2227221F821B71
:1011F0009109681B888199810E94440797B5898568
:101200008917B1F067B527B5281B330B81E090E053
:101210001216130614F090E080E0232F221F2227DD
:10122000221F821B9109681B888199810E943E07B9
:101230009091B4008A85891731F16091B4002091B2
:10124000B400281B330B81E090E01216130614F053
:1012500090E080E0232F221F2227221F821B91096A
:10126000681B8A819B81DF91CF910C94440769852B
:10127000888199810E943E076885888199810E94B2
:1012800044076A85EECFDF91CF91089588B5089520
:101290008091B400089587B50895EE0FFF1F059063
:1012A000F491E02D0994A0E0B0E0E9E5F9E00C94B8
:1012B000800D5C016B017A016115710519F0FB016C
:1012C00091838083E114F10429F0C7010297839789
:1012D00008F0E5C0E5012196F5011081812F90E02D
:1012E0000E94870A892B11F05E01F4CF1D3229F488
:1012F0002196F501118101E007C01B3221F4E501BF
:101300002296F501118100E0E114F10409F1F0E108
:10131000EF16F10429F43FC010E3E114F10421F1C8
:1013200028E0E216F10401F154F4E2E0EE16F104D3
:1013300021F5812C912CA12CB0E4BB2E3EC0FAE00B
:10134000EF16F10439F020E1E216F104B1F430C0F7
:10135000103319F1FAE0EF2EF12CACEC8A2E982C18
:10136000A82CACE0BA2E29C078E0E72EF12C812C15
:10137000912CA12CE0E1BE2E20C060E070E080E066
:1013800090E897010F2C000C440B550B0E94520D56
:1013900049015A0112C0103359F488818F7D883574
:1013A00009F0BACF19812296026080E1E82EF12C73
:1013B000812C912CA12C68E0B62E40E060E070E01A
:1013C000CB0127010F2C000C66087708FE0150EDB9
:1013D000352E310E29E0231570F42FEB210F2A3121
:1013E00018F439EC332E06C02FE9210F2A3118F5F5
:1013F00029EA322E310E232D30E02E153F05DCF484
:1014000047FD16C086169706A806B90670F0A30118
:1014100092010E94420D630D711D811D911D61306D
:101420007105810520E8920710F04FEF01C041E0FF
:1014300021961081CBCF202F2170C114D10471F0DF
:10144000442329F02197F601D183C08307C001FF0F
:1014500019C02297F601D183C08314C047FF12C080
:10146000222329F060E070E080E090E804C06FEF94
:101470007FEF8FEF9FE722E230E030932307209346
:10148000220709C0222381F090958095709561957F
:101490007F4F8F4F9F4F462F372F282F12C040E08E
:1014A00030E020E090E00DC097FFF5CF82E290E0C1
:1014B00090932307809322076FEF7FEF8FEF9FE7D3
:1014C000EACF642F732F822FCDB7DEB7E1E10C9402
:1014D0009C0DFC0188279927E89421912032E9F39B
:1014E000293010F02E30C8F32B3241F02D3239F470
:1014F000689404C00E949E0A820F911D219120537E
:101500002A30C0F31EF4909581959F4F0895911154
:101510000C949B0C803219F089508550C8F70895BF
:10152000FB01DC014150504030F08D910190801959
:1015300019F40020B9F7881B990B08957AE0979F5A
:10154000902D879F802D910D11240895AEE0B0E07D
:10155000ECEAFAE00C948D0D0D891E8986E08C83EF
:101560001A8309838FEF9FE79E838D83AE01475EC9
:101570005F4F6F89788DCE0101960E94C80AEF8176
:10158000F885E00FF11F10822E96E4E00C94A90D6F
:10159000ACE0B0E0EEECFAE00C947F0D6C017B0166
:1015A0008A01FC0117821682838181FFBEC1CE01B0
:1015B00001964C01F6019381F70193FD859193FF0C
:1015C00081917F01882309F4ACC1853239F493FD00
:1015D000859193FF81917F01853229F4B60190E0D6
:1015E0000E94B40CE7CF512C312C20E02032A0F423
:1015F0008B3269F030F4803259F0833269F4206123
:101600002CC08D3239F0803339F4216026C022603D
:10161000246023C0286021C027FD27C030ED380F8B
:101620003A3078F426FF06C0FAE05F9E300D1124B0
:10163000532E13C08AE0389E300D1124332E2062C1
:101640000CC08E3221F426FD6CC1206406C08C369D
:1016500011F4206802C0883641F4F70193FD8591AA
:1016600093FF81917F018111C1CF982F9F7D955468
:10167000933028F40C5F1F4F9FE399830DC083368E
:1016800031F0833771F0833509F05BC022C0F80177
:10169000808189830E5F1F4F44244394512C540151
:1016A00015C03801F2E06F0E711CF801A080B18006
:1016B00026FF03C0652D70E002C06FEF7FEFC5010C
:1016C0002C870E94A90C2C0183012C852F77222EB8
:1016D00017C03801F2E06F0E711CF801A080B180D4
:1016E00026FF03C0652D70E002C06FEF7FEFC501DC
:1016F0002C870E949E0C2C012C852068222E8301B1
:1017000023FC1BC0832D90E048165906B0F4B601A7
:1017100080E290E00E94B40C3A94F4CFF50127FCEB
:10172000859127FE81915F01B60190E00E94B40C83
:1017300031103A94F1E04F1A51084114510471F7F5
:10174000E6C0843611F0893639F5F80127FF07C065
:1017500060817181828193810C5F1F4F08C060811D
:101760007181072E000C880B990B0E5F1F4F2F768F
:10177000722E97FF09C090958095709561957F4F67
:101780008F4F9F4F2068722E2AE030E0A4010E9404
:10179000E40CA82EA81844C0853729F42F7EB22E59
:1017A0002AE030E025C0F22FF97FBF2E8F36C1F03E
:1017B00018F4883579F0B5C0803719F0883721F0F2
:1017C000B0C02F2F2061B22EB4FE0DC08B2D8460CF
:1017D000B82E09C024FF0AC09F2F9660B92E06C0FC
:1017E00028E030E005C020E130E002C020E132E036
:1017F000F801B7FE07C060817181828193810C5F1F
:101800001F4F06C06081718180E090E00E5F1F4F26
:10181000A4010E94E40CA82EA818FB2DFF777F2EB0
:1018200076FE0BC0372D3E7FA51450F474FE0AC01F
:1018300072FC08C0372D3E7E05C0BA2C372D03C080
:10184000BA2C01C0B52C34FF0DC0FE01EA0DF11D0C
:101850008081803311F4397E09C032FF06C0B39411
:10186000B39404C0832F867809F0B39433FD13C07A
:1018700030FF06C0B31498F43A0C532C5B1810C018
:10188000B31470F4B60180E290E03C870E94B40C7F
:10189000B3943C85F5CFB31418F43B1802C05A2C0E
:1018A000312C34FF12C0B60180E390E03C870E94E7
:1018B000B40C3C8532FF17C031FD03C088E790E0CF
:1018C00002C088E590E0B6010CC0832F867859F0FD
:1018D00031FF02C08BE201C080E237FD8DE2B6012C
:1018E00090E00E94B40CA51438F4B60180E390E0B7
:1018F0000E94B40C5A94F7CFAA94F401EA0DF11D9A
:101900008081B60190E00E94B40CA110F5CF332085
:1019100009F450CEB60180E290E00E94B40C3A94F3
:10192000F6CFF6018681978102C08FEF9FEF2C964C
:10193000E2E10C949B0D992788270895FC010590FE
:10194000615070400110D8F7809590958E0F9F1FC1
:101950000895FC016150704001900110D8F7809506
:1019600090958E0F9F1F08950F931F93CF93DF9332
:10197000182F092FEB018B8181FD03C08FEF9FEFA3
:101980001EC082FF0FC02E813F818C819D81281750
:10199000390774F4E881F981CF010196998388832E
:1019A000108306C0E885F985812F0995892B31F7C9
:1019B0008E819F8101969F838E83812F902FDF914F
:1019C000CF911F910F910895FA01AA27283051F164
:1019D000203181F1E8946F936E7F6E5F7F4F8F4F60
:1019E0009F4FAF4FB1E03ED0B4E03CD0670F781FBF
:1019F000891F9A1FA11D680F791F8A1F911DA11DA4
:101A00006A0F711D811D911DA11D20D009F46894DC
:101A10003F912AE0269F11243019305D3193DEF684
:101A2000CF010895462F4770405D4193B3E00FD03A
:101A3000C9F7F6CF462F4F70405D4A3318F0495D25
:101A400031FD4052419302D0A9F7EACFB4E0A69508
:101A50009795879577956795BA95C9F7009761052A
:101A6000710508959B01AC010A2E06945795479580
:101A700037952795BA95C9F7620F731F841F951F75
:101A8000A01D0895DB018F939F930E94740DBF9159
:101A9000AF91A29F800D911DA39F900DB29F900DBD
:101AA00011240895A1E21A2EAA1BBB1BFD010DC033
:101AB000AA1FBB1FEE1FFF1FA217B307E407F507FE
:101AC00020F0A21BB30BE40BF50B661F771F881FDA
:101AD000991F1A9469F760957095809590959B0170
:101AE000AC01BD01CF0108950E94B60DA59F900DD8
:101AF000B49F900DA49F800D911D112408952F92E5
:101B00003F924F925F926F927F928F929F92AF928D
:101B1000BF92CF92DF92EF92FF920F931F93CF93DA
:101B2000DF93CDB7DEB7CA1BDB0B0FB6F894DEBF71
:101B30000FBECDBF09942A88398848885F846E8497
:101B40007D848C849B84AA84B984C884DF80EE80E1
:101B5000FD800C811B81AA81B981CE0FD11D0FB6EA
:101B6000F894DEBF0FBECDBFED010895A29FB00176
:101B7000B39FC001A39F700D811D1124911DB29FC1
:0E1B8000700D811D1124911D0895F894FFCF62
:101B8E006164640052656C617920736176656421CD
:101B9E00204E554D4245523A2025752049443A2053
:101BAE0025580A0055736167653A2072656C617934
:101BBE0020616464205B69645D202020205B696481
:101BCE005D206265696E672061203136626974201E
:101BDE00686578206E756D6D6265720A006C69734A
:101BEE00740052656C6179733A0A0052454C415942
:101BFE003A202575207475726E6564206F6E0A002A
:101C0E004E6F2073757463682052656C61790A009B
:101C1E0052454C41593A202575207475726E656493
:101C2E00206F66660A00206973206E6F7420612033
:101C3E0076616C696420737562636F6D6D616E643D
:101C4E003A2072656C6179205B6164642F6C6973F4
:101C5E00742F6F6E2F6F66665D0A00524742206CBE
:101C6E006967687473206F6E0A00524742206C6970
:101C7E0067687473206F66660A007072696E74000E
:101C8E0043757272656E74205247422076616C7590
:101C9E0065733A0A523A20257520473A2025752059
:101CAE00423A2025750A0053657420524742207629
:101CBE00616C7565730A0055736167653A207267CA
:101CCE006220736574205B5252525D205B4747471A
:101CDE005D205B4242425D0A007061747465726EF3
:101CEE0000536574205061747465726E0A007072D0
:101CFE006573657400536574205072657365740A5C
:101D0E000066616465206F6E005475726E656420A6
:101D1E006F6E20466164650A0066616465206F66B9
:101D2E0066005475726E6564206F66662046616447
:101D3E00650A00206973206E6F7420612076616CD5
:101D4E00696420737562636F6D6D616E643A2072A3
:101D5E006762205B2F6F6E2F6F66662F7072696ED3
:101D6E00742F7365742F7061747465726E2F707238
:101D7E00657365745D0A0072656C617900726762E5
:101D8E0000657261736500454550524F4D20657276
:101D9E00617365640A0068656C7000417661696CF8
:101DAE0061626C6520436F6D6D616E64733A200ADB
:101DBE002020202020202020202020202020202015
:101DCE0068656C70202020202020202020202020DC
:101DDE0020202020202020202020203A2020536860
:101DEE006F7720746869732070726F6D7074200A3B
:101DFE0020202020202020202020202020202020D5
:101E0E0072656C617920616464205B69645D202079
:101E1E0020202020202020202020203A2020416435
:101E2E006420576972656C6573732052656C6179B5
:101E3E000A202020202020202020202020202020AA
:101E4E002072656C6179206C6973742020202020CB
:101E5E002020202020202020202020203A2020502A
:101E6E0072696E74206C697374206F66207361766C
:101E7E00656420576972656C6573732052656C6179
:101E8E007973200A202020202020202020202020AE
:101E9E002020202072656C6179205B6F6E2F6F663B
:101EAE00665D205B6E6E5D20202020202020203A73
:101EBE0020205475726E206F6E2F6F6666206E74C2
:101ECE00682072656C61790A202020202020202055
:101EDE002020202020202020657261736520202084
:101EEE0020202020202020202020202020202020E4
:101EFE002020203A20204572617365206570707233
:101F0E006F6D0A202020202020202020202020203D
:101F1E00202020726762205B6F6E2F6F66665D20D9
:101F2E0020202020202020202020202020203A2089
:101F3E00205475726E206F6E2F6F66662052474268
:101F4E00206C6564732061742063757272656E74A3
:101F5E002076616C75652E0A2020202020202020FE
:101F6E002020202020202020726762207072696E4F
:101F7E0074202020202020202020202020202020FF
:101F8E002020203A20205072696E74206375727280
:101F9E00656E74205247422076616C75652E0A205C
:101FAE0020202020202020202020202020202072D1
:101FBE00676220736574205B5252525D205B474707
:101FCE00475D205B4242425D20203A2020536574DB
:101FDE00205247422076616C75652C2070617474B6
:101FEE0065726E206D75737420626520302E0A2026
:101FFE002020202020202020202020202020207281
:10200E006762207061747465726E205B69645D2016
:10201E00202020202020202020203A20205247421D
:10202E00207061747465726E0A202020202020209A
:10203E0020202020202020202072676220707265D0
:10204E00736574205B69645D202020202020202091
:10205E00202020203A2020736574207072657365ED
:10206E007420636F6C6F720A2020202020202020A5
:10207E002020202020202020726762206661646567
:10208E00205B6F6E2F6F66665D2020202020202043
:10209E002020203A20207475726E20436F6C6F7270
:1020AE0066616465206F6E206F72206F66660A200F
:1020BE0020202020202020202020202020202076BC
:1020CE00657273696F6E2020202020202020202032
:1020DE00202020202020202020203A20205072690D
:1020EE006E742056657273696F6E2E0A004E6F7491
:1020FE0020612076616C696420636F6D6D616E6422
:10210E000A00524742436F6E74726F6C6C65722098
:10211E0076302E33207374617274696E670A000014
:00000001FF
